:1000000009298030A100FE30A7200130A7207530DB
:10001000A7003030BE28A101A117AF00AF08031D13
:100020001328030114280130AF020310A20CA20C04
:10003000A20CC0302205403EAF07FE30A7202F089B
:10004000A728A101A117AF00FE30A7202F08A728DD
:10005000A401AA00AB01A01124080319A0150530C2
:10006000A3002730A900103041200330A900E83058
:100070004120A90164304120A9010A3041202A0809
:100080004828A8002B08A7002A08A600D220260886
:10009000A600A3030319A011240803195228230260
:1000A000031859282608031DA011A0195928303E0D
:1000B000A7280800AD0006118611831606118611C7
:1000C0000F30860583122D08A01884283E30A70023
:1000D0008030BE203330AC0098201330A700883029
:1000E000BE2098206430BD2098206430BD2022308E
:1000F000AC009820283083200C30832006308320E9
:10010000A0142D0884282014AC00201C92288611ED
:10011000033C031C972897200530A700DC30BE2045
:10012000031408002014FE3C0319A5288615201C82
:10013000201006150F3086052C08F03986040611AC
:10014000AC0E201898283230BD202D080429A11BA0
:100150005A2883178001840AFF3E031DAA28042918
:10016000A901A800FF30A807031CA907031C042944
:100170000330A700DF30BE20B228A701E83EA6006A
:10018000A709FC30031CC728A6070318C428A60724
:100190000000A70FC4282618CD28A61CD1280000CF
:1001A000D1280800AB01AA011030AC00270DAA0D20
:1001B000AB0D2808AA022908031C290FAB0203185B
:1001C000E8282808AA0729080318290FAB070310F5
:1001D000A60DA70DAC0BD628260804291030B000B8
:1001E000A701A601AD0CAC0C031CFC282808A6072F
:1001F00029080318290FA707A70CA60CAB0CAA0CFB
:10020000B00BF2282A080429831383120313000079
:100210000800A00107309F00E03083168500FF3002
:1002200086008113831285018601203084006030AE
:10023000AA20A03084005030AA2020308400303022
:10024000A920C830B020012077305A205A205A20E7
:100250002E305A2070305A2069305A2063305A208C
:1002600062305A2061305A2073305A2069305A2047
:1002700063305A202E305A206E305A206C305A206B
:100280000B30A900B830B120012044305A2043304F
:100290005A2046305A2032305A2030305A205530B9
:1002A0005A204B305A2042305A2020305A205A20AF
:1002B00056305A202D305A2032305A200730A900AB
:1002C000D030B120012041305A2064305A206A30A9
:1002D0005A2075305A2073305A2074305A202030FA
:1002E0005A204C305A2044305A2052305A20861816
:1002F0007F29851F7D2905147E2905107729012076
:1003000053305A2065305A2061305A2072305A20BA
:1003100063305A2068305A2020305A2073305A20D7
:1003200069305A2067305A206E305A2061305A2086
:100330006C305A20361405128316051283122D2AAA
:10034000C3013C03A500C90149082502031CB929C2
:10035000DC21B61CB7294308A6004908A200A60163
:10036000A20A0314A60DA20BB2292608C304C90FC2
:10037000A429B2014308B100B20CB10CB20CB10C0B
:10038000B20CB10CB20CB10C0F30B2053208AD009A
:100390003108AC00A9010A30A800EE20B1002B08FA
:1003A000B200B4014308B3000F30B3050030B40508
:1003B00031083307C3000800BA01B9010618F12952
:1003C0000130B020B90A0319BA0A0B303A02031CF3
:1003D000F029031DEF29B9303902031CF0296F2CD5
:1003E000DE299B30B0200618B614061CB610361C49
:1003F0000D2AAD014408AC00A9011430A800EE207C
:10040000B1002B08B2003208A7003108A600A901EC
:100410003A30A800D220BD00202A8030A10001304F
:10042000A2003D080D200230A40044082920030149
:100430003619013EB618013A03193611031D361557
:10044000C40A85140130A900F430B1208510A90137
:10045000F030A8002808B1200800BB01C401361202
:10046000361AC52ABA01B901061C472AB90A031966
:10047000BA0A0130B020AF303A02031C462A031DED
:10048000452AC9303902031C462A6F2C342ABA0186
:10049000B9010618832AB90A0319BA0A0A30B0202A
:1004A0003618772A39080B3A3A04031D622A80303D
:1004B000A1000130A2003D080D2035305A2039300E
:1004C0005A20762A3908193A3A04031D692A8514F4
:1004D000762A39084B3A3A04031D702A8510762A89
:1004E0003908FA3A3A04031D762A6F2C822A113011
:1004F0003A02031C822A031D812A95303902031C0B
:10050000822A6F2C492A41303B02031C882A6F2C17
:10051000BB0A3A08031D902A65303902031C912A50
:100520003616361CC42AAD013B08AC00A9011430B4
:10053000A800EE20B1002B08B2003208A700310855
:10054000A600A9014130A800D220BD008030A10042
:100550008030212046305A206F305A2075305A2082
:100560006E305A2064305A2020305A2073305A207E
:1005700069305A2067305A206E305A2061305A2034
:100580006C305A2020305A20302A361CE12A0120B3
:1005900049305A206E305A2069305A2074305A201F
:1005A00069305A2061305A206C305A2069305A2004
:1005B0007A305A2065305A202E305A205A205A203C
:1005C000502B0B30BD000130A2003D080B20A101D3
:1005D000B61DF92A3B3041020318F02AC10AF82A55
:1005E000C101173045020318F72AC50AF82AC501C8
:1005F000FD2A4208C1004608C500051B0D2B450811
:10060000031D052B0C30C7000C2B0D304502031CBD
:100610000C2B0C304502C700122B4508C7002030B8
:100620005A205A200A3047020318182B20305A202B
:100630008030A100470828203A305A200230A40018
:10064000410829203A305A2030305A205A20051BC0
:10065000392B0C3045020318322B61305A206D3093
:100660005A20362B70305A206D305A201130BD0080
:100670003B2B1330BD00410803190130031D03015A
:10068000B5001E30410203190130031D030135047A
:10069000B50001308618030135040319502B472C8F
:1006A000361E452CDC210130C9000F3049020318E9
:1006B0005C2BDC21C90F552B3611B611DC21DC2156
:1006C000DC21B61C652B0514662B05101230C90001
:1006D0001430490203186F2BDC21C90F682BDC2171
:1006E0000730BC00A0214308C200DC21361D792B55
:1006F000B6150630BC00A0214308C600DC21361D1B
:10070000822BB6150630BC00A0214308BE00033082
:10071000BC00A0214308C8000530BC00A02143084C
:10072000C0000830BC00A0214308BF00DC21361DFA
:100730009A2BB615361CA02BB6199F2B361001200C
:10074000B619442C8030A100803021203E0828209A
:1007500020305A2001304002031DB52B4A305A2068
:1007600061305A206E305A202D2C02304002031D79
:10077000C02B46305A2065305A2062305A202D2C2A
:1007800003304002031DCB2B4D305A2061305A20DC
:1007900072305A202D2C04304002031DD62B4130DC
:1007A0005A2070305A2072305A202D2C05304002C9
:1007B000031DE12B4D305A2061305A2079305A20E8
:1007C0002D2C06304002031DEC2B4A305A20753088
:1007D0005A206E305A202D2C07304002031DF72B73
:1007E0004A305A2075305A206C305A202D2C08304F
:1007F0004002031D022C41305A2075305A206730C8
:100800005A202D2C09304002031D0D2C53305A2044
:1008100065305A2070305A202D2C0A304002031DBA
:10082000182C4F305A2063305A2074305A202D2C07
:100830000B304002031D232C4E305A206F305A20BB
:1008400076305A202D2C0C304002031D2D2C4430C4
:100850005A2065305A2063305A20051B3A2C20302C
:100860005A208030A1000230A4003F082920203007
:100870005A20442C20305A2027305A208030A100A2
:100880000230A4003F082920462C6F2C2D2A851FFA
:100890004E2C0512831605128312502C8316051652
:1008A00083129B30B020410803190130031D03015E
:1008B000B50001308618030135040319602C0515B5
:1008C000851585140130A900F430B120051185117A
:1008D00085100130A9004A30B120C40A532B0120F1
:1008E0004E305A206F305A2020305A2073305A2010
:1008F00069305A2067305A206E305A2061305A20B1
:100900006C305A20203084006030AA20A03084004F
:100910005030AA20203084003030A9200618B616A6
:10092000061CB61203010618013EB61A013C031D4F
:100930009F2CB70A0319B80A0130B020922C03018A
:10094000B61A0130013A0319B612031DB616030197
:100950000618013EB61A013C031DB42CB70A031950
:10096000B80A0130B020A72C03303802DE3003195A
:0A09700037020318822C36142D2ADA
:02400E00503F21
:00000001FF
